:020000040800F2
:10000000000900202D080008B11C0008811C000810
:100010009D1C0008811C0008951C00082F08000882
:100020002F0800082F0800082F080008E5370008EF
:100030002F0800082F0800082F080008F93C0008C6
:100040002F0800082F0800082F0800082F080008B4
:100050002F0800082F080008293A0008553A000820
:10006000813A0008AD3A0008D93A00082F08000884
:100070002F0800082F0800082F0800082F08000884
:100080002F0800082F0800082F080008AD2C0008D2
:10009000192D00086D2D0008C12D0008053B000832
:1000A0002F0800082F0800082F0800082F08000854
:1000B0002F0800082F0800082F0800082F08000844
:1000C0002F0800082F0800082F0800082F08000834
:1000D0002F0800082F0800082F0800082F08000824
:1000E0006D3B00082F0800082F0800082F080008A3
:1000F0002F0800082F0800082F0800082F08000804
:100100002F0800082F0800082F0800082F080008F3
:100110002F0800082F0800082F0800082F080008E3
:100120002F0800082F0800082F0800082F080008D3
:100130002F0800082F0800082F0800082F080008C3
:100140002F0800082F0800082F0800082F080008B3
:100150002F0800082F0800082F0800082F080008A3
:100160004FF0FF0C1CEAD0521EBF1CEAD15392EA9A
:100170000C0F93EA0C0F6FD01A4480EA010C400276
:1001800018BF5FEA41211ED04FF0006343EA5010D0
:1001900043EA5111A0FB01310CF00040B1F5000F12
:1001A0003EBF490041EAD3715B0040EA010062F1C1
:1001B0007F02FD2A1DD8B3F1004F40EBC25008BFAB
:1001C00020F00100704790F0000F0CF0004C08BFC9
:1001D00049024CEA502040EA51207F3AC2BFD2F196
:1001E000FF0340EAC250704740F400004FF00003A4
:1001F000013A5DDC12F1190FDCBF00F000407047DE
:10020000C2F10002410021FA02F1C2F1200200FA1B
:1002100002FC5FEA310040F1000053EA4C0308BFE2
:1002200020EADC70704792F0000F00F0004C02BF33
:10023000400010F4000F013AF9D040EA0C0093F0AE
:10024000000F01F0004C02BF490011F4000F013B08
:10025000F9D041EA0C018FE70CEAD15392EA0C0F76
:1002600018BF93EA0C0F0AD030F0004C18BF31F0E1
:10027000004CD8D180EA010000F00040704790F0B7
:10028000000F17BF90F0004F084691F0000F91F05B
:10029000004F14D092EA0C0F01D142020FD193EA21
:1002A0000C0F03D14B0218BF084608D180EA0100A9
:1002B00000F0004040F0FE4040F40000704740F085
:1002C000FE4040F44000704780F0004002E000BF74
:1002D00081F0004142001FBF5FEA410392EA030F31
:1002E0007FEA226C7FEA236C6AD04FEA1262D2EB7B
:1002F0001363C1BFD218414048404140B8BF5B4280
:10030000192B88BF704710F0004F40F4000020F018
:100310007F4018BF404211F0004F41F4000121F02E
:100320007F4118BF494292EA030F3FD0A2F1010278
:1003300041FA03FC10EB0C00C3F1200301FA03F1B6
:1003400000F0004302D5494260EB4000B0F5000FD9
:1003500013D3B0F1807F06D340084FEA310102F198
:100360000102FE2A51D2B1F1004F40EBC25008BF4A
:1003700020F0010040EA03007047490040EB000014
:10038000013A28BFB0F5000FEDD2B0FA80FCACF115
:10039000080CB2EB0C0200FA0CF0AABF00EBC25042
:1003A00052421843BCBFD0401843704792F0000F30
:1003B00081F4000106BF80F400000132013BB5E783
:1003C0004FEA41037FEA226C18BF7FEA236C21D0F9
:1003D00092EA030F04D092F0000F08BF084670475E
:1003E00090EA010F1CBF0020704712F07F4F04D12C
:1003F000400028BF40F00040704712F100723CBF3F
:1004000000F50000704700F0004343F0FE4040F468
:10041000000070477FEA226216BF08467FEA236326
:100420000146420206BF5FEA412390EA010F40F411
:10043000800070474FF0000304E000BF10F000435D
:1004400048BF40425FEA000C08BF704743F0964344
:1004500001464FF000001CE050EA010208BF70475F
:100460004FF000030AE000BF50EA010208BF7047E6
:1004700011F0004302D5404261EB41015FEA010CFB
:1004800002BF84460146002043F0B64308BFA3F1F3
:100490008053A3F50003BCFA8CF2083AA3EBC253D5
:1004A00010DB01FA02FC634400FA02FCC2F12002F4
:1004B000BCF1004F20FA02F243EB020008BF20F02B
:1004C0000100704702F1200201FA02FCC2F1200291
:1004D00050EA4C0021FA02F243EB020008BF20EA86
:1004E000DC70704742000ED2B2F1FE4F0BD34FF0DA
:1004F0009E03B3EB126209D44FEA002343F000439A
:1005000023FA02F070474FF00000704712F1610FBC
:1005100001D1420202D14FF0FF3070474FF000008E
:10052000704700BF53B94AB9002908BF00281CBF53
:100530004FF0FF314FF0FF3000F076B9ADF1080C0D
:100540006DE904CE00F006F8DDF804E0DDE90223F1
:1005500004B070472DE9F047089E0D4604468846D2
:10056000002B4DD18A42944668D9B2FA82F252B138
:1005700001FA02F3C2F1200120FA01F10CFA02FCA7
:1005800041EA030894404FEA1C41B8FBF1F71FFA17
:100590008CFE01FB178807FB0EF0230C43EA08438F
:1005A00098420AD91CEB030307F1FF3580F01E8146
:1005B000984240F21B81023F63441B1AB3FBF1F0E7
:1005C00001FB103300FB0EFEA4B244EA0344A6452F
:1005D0000AD91CEB040400F1FF3380F00981A64521
:1005E00040F20681644402380021A4EB0E0440EA84
:1005F00007401EB10023D440C6E90043BDE8F087A0
:100600008B4208D9002E00F0EE800021C6E90005DB
:100610000846BDE8F087B3FA83F100294AD1AB421E
:1006200002D3824200F2FC80841A65EB03030120AE
:100630009846002EE2D0C6E90048DFE702B9FFDEA7
:10064000B2FA82F2002A40F09180A1EB0C00012165
:100650004FEA1C471FFA8CFEB0FBF7F307FB1300B1
:10066000250C45EA00450EFB03F0A84208D91CEB17
:10067000050503F1FF3802D2A84200F2CE804346BE
:100680002D1AB5FBF7F007FB10550EFB00FEA4B2C8
:1006900044EA0544A64508D91CEB040400F1FF35E3
:1006A00002D2A64500F2B6802846A4EB0E0440EA2A
:1006B00003409EE7C1F120078B4022FA07FC4CEA79
:1006C000030C25FA07FA4FEA1C49BAFBF9F820FA9D
:1006D00007F309FB18AA8D401FFA8CFE1D4300FA90
:1006E00001F308FB0EF02C0C44EA0A44A04202FA83
:1006F00001F20BD91CEB040408F1FF3A80F088806A
:10070000A04240F28580A8F102086444241AB4FB98
:10071000F9F009FB104400FB0EFEADB245EA0444BB
:10072000A64508D91CEB040400F1FF356CD2A645A0
:100730006AD90238644440EA0840A0FB0295A4EB61
:100740000E04AC42C846AE4656D353D0002E69D0F4
:10075000B3EB080264EB0E0422FA01F304FA07F784
:100760001F43CC40C6E90074002147E70CFA02FCA5
:10077000C2F1200125FA01F34FEA1C4720FA01F1EA
:1007800095400D43B3FBF7F107FB11331FFA8CFEC5
:10079000280C40EA034001FB0EF3834204FA02F402
:1007A00008D91CEB000001F1FF382FD283422DD96C
:1007B00002396044C01AB0FBF7F307FB1300ADB277
:1007C00045EA004503FB0EF0A84208D91CEB0505DD
:1007D00003F1FF3816D2A84214D9023B6544281A07
:1007E00043EA014138E73146304607E72F46E4E661
:1007F0001846F9E64B45A9D2B9EB020865EB0C0E99
:100800000138A3E74346EAE7284694E74146D1E7A3
:10081000D0467BE76444023847E7023B65442FE754
:10082000084606E73146E9E6704700BF02E000F0FF
:1008300000F8FEE772B6264880F30888254880F362
:100840000988254825490860022080F31488BFF3F1
:100850006F8F03F017F803F07BF84FF05530204905
:100860001B4A91423CBF41F8040BFAE71D49194A63
:1008700091423CBF41F8040BFAE71B491B4A1C4B51
:100880009A423EBF51F8040B42F8040BF8E70020EF
:100890001849194A91423CBF41F8040BFAE702F0AB
:1008A000F5FF03F057F8154C154DAC4203DA54F838
:1008B000041B8847F9E700F03FF8124C124DAC4298
:1008C00003DA54F8041B8847F9E702F0DDBF0000A3
:1008D00000090020001100200000000808ED00E0E1
:1008E0000001002000090020103E00080011002037
:1008F0002411002028110020E025002060010008BC
:100900006001000860010008600100082DE9F04F57
:10091000C1F80CD0C3689D46BDE8F08F002383F377
:1009200011882846A047002002F010FDFEE702F0E3
:1009300083FC00DFFEE70000F8B500F03DFE02F0AA
:10094000EFFE074602F03AFF0546002840D12C4B47
:100950009F423DD001339F423DD02A4B27F0FF02FA
:100960009A423BD1F8B200F003FC2E4642F21074DA
:1009700000F004FC08B10024264601F007F988B312
:100980000024032000F044F8264635B11E4B9F4258
:1009900003D0002402F00AFF2646002002F0CAFE1F
:1009A0001A4B9B6813F0400322D00EB100F046F8BA
:1009B00000F044FC00F002FE01F07CF90546CCB1E9
:1009C00001F078F9401BA04214D900F037F8F3E7A2
:1009D0002E460024CCE704460126C9E706464FF41C
:1009E0007A74C5E7002CD0D04FF47A740126CCE796
:1009F0001C46DDE700F0D4FC012002F0ADFCDEE790
:100A0000010007B0000008B0263A09B0000C014010
:100A1000084B187003280CD8DFE800F0080502081E
:100A2000022000F027BE022000F01CBE0022024B74
:100A30005A607047281100202C11002038B501F0B1
:100A4000A5F830B103221F4B1A7000221E4B5A60CA
:100A500038BD1E4B1E4A19680131F9D00433934248
:100A6000F9D11C4C194DD4F80424AA42F0D31A4BE6
:100A70009B6803F1006303F5C8439A42E8D202F091
:100A800069FE02F07BFE002000F0B2FD0220FFF7BD
:100A9000BFFF124BDA690022DA61D96999699A615C
:100AA0009B6972B64FF0E023C3F8085D3021D4F89B
:100AB0000034D4F8042481F311889D4683F3088818
:100AC0001047C5E7281100202C1100200064000801
:100AD000206400080060000800110020001002409F
:100AE00049F26900084A136899B21B0C00FB0133F4
:100AF00044F250611360054B186882B2000C01FB90
:100B00000200186080B27047201100201C110020E4
:100B100010B504460021102200F0C8FD034B03CBA2
:100B2000206061601868A06010BD00BFE8F7FF1F7B
:100B30002DE9F0410026ADF5507D6EAC40F2751206
:100B400007460D4610A831460F9600F0AFFD4FF452
:100B5000C4723146204600F0A9FD01F0ABF84FF415
:100B60007A72B0FBF2F0264B0DF13C08186093E866
:100B70000700022384E807000DF5ED702382FFF7DC
:100B8000C7FF4EF603031F4907A8238403F0ECF8C0
:100B90001F230DF2EB2284F832310DF1340C07AB38
:100BA0001E4603CE664510605160334602F10802CE
:100BB000F6D130681060B188B37920469180937186
:100BC0004146012200F0BEFD00230393AB7E80B2BC
:100BD000029305F1190301930123CDE904800093E9
:100BE000384605A3D3E90023E97E01F0A9FB0DF502
:100BF000507DBDE8F08100BF9E6AC421818A46EE27
:100C000034110020783D00082DE9F041264D804642
:100C10002B7A0C46DAB0FBB9204627A900F0A2FED9
:100C20000746002836D19DF89D60C82E32D801466F
:100C30004FF4FA72284600F039FD32460DF19E015C
:100C400005F1090000F020FD9DF89C302E447772DC
:100C50002B720BB9E37E2B728122002106AD27A8EF
:100C600000F024FD0122294627A800F0B7FE00234A
:100C70000393A37E80B2029304F119030193282306
:100C8000CDE904500093404605A3D3E90023E17E5B
:100C900001F056FB5AB0BDE8F08100BFAFF3008011
:100CA00026417272DF25D7B77C210020F0B54FF4C2
:100CB0008A750024234EF1B005FB006596F8D83004
:100CC000D822214685F8DC3085F8E8403AA800F0C3
:100CD000EDFC06F1090000F0E1FCD5F8E430C2B209
:100CE00006AF8DF8F00006F109010DF1F100CDE934
:100CF0003A3400F0C9FC394601223AA800F09AFEC5
:100D000080B2CDE9047008230127CDE9023706F14E
:100D1000D80301933023317A00930B4807A3D3E91A
:100D2000002301F00DFBA04206DD00F0C3FFC5F873
:100D3000E000384671B0F0BD2046FBE778F6339FFF
:100D400093CACD8D7C2100204C210020F0B51E4E91
:100D50001E4F1F4D85B0304601F01EFB044660B3A8
:100D600010220021684600F0A1FC4FF00003227B16
:100D70006068A16862F303038DF8003002AB03C31F
:100D8000019B2268384662F31C0301939DF80030F2
:100D90006A4643F020038DF800300023194602F024
:100DA00087F9044620B9304601F0FAFA2C70D2E7F0
:100DB0002B78072B03D801332B7005B0F0BD024808
:100DC00001F0EEFAF9E700BF4C210020A823002033
:100DD0007523002070B50D4614461E4601F00CFA2E
:100DE00050B9022E10D1012C0ED112A3D3E9002349
:100DF0000120C5E9002307E0282C10D005D8012CDC
:100E000009D0052C0FD0002070BD302CFBD10BA3D6
:100E1000D3E90023ECE70BA3D3E90023E8E70BA316
:100E2000D3E90023E4E70BA3D3E90023E0E700BF05
:100E3000AFF30080401DA12026812A0B78F6339F56
:100E400093CACD8D9E6AC421818A46EE2641727274
:100E5000DF25D7B7F017304A39059E5638B5054615
:100E60000E4C0021013500F0E5FBA4F8F051B4F878
:100E7000F00100F0C7FB78B1B4F8F00100F0D2FB4C
:100E8000014648B9B4F8F00100F0D4FBB4F8F031F1
:100E90000133A4F8F031EAE738BD00BF7C2100201F
:100EA0002DE9F04F8DB000AF04460D4601F0A4F9D6
:100EB000002846D12B7E022B1AD1EB8A012B17D1A9
:100EC00000F0F8FE0646FFF70BFE4FF4C873B0FBC8
:100ED000F3F202FB1303DFF878829BB206F5167675
:100EE0003344C8F80030EB7E33B90022994B1A70B6
:100EF0003437BD46BDE8F08F284607F11C0100F0ED
:100F0000EFFC0028F4D107F10C00FFF701FEBD7FD4
:100F100007F10C012A4607F11F0002F0F5FE002838
:100F2000E3D10F2D08D88B4B1D70D8F80030A3F5F6
:100F30001673C8F80030DBE72046397F01F054F91A
:100F4000D6E7EB8A282B6BD010D8012B63D0052B6A
:100F5000CED1BFF34F8F8049804BCA6802F4E06264
:100F60001343CB60BFF34F8F00BFFDE7302BBFD1E2
:100F70007B4CEA7E237A9A42BAD194F8DC206B7ECD
:100F80009A42B5D1284604F1EA0100F07FFD0646F9
:100F90000028ADD1012384F8E83000F08BFED4F8AE
:100FA000E030C01A192840F6B83338BF19209842EB
:100FB00028BF1846FFF73EFA6A49FFF7D1F8054601
:100FC0002068FFF737FA6849FFF7CAF80146284654
:100FD000FFF780F9FFF786FA20604FF48A7194F8E2
:100FE000D9307B607A68636801FB02F5621992F878
:100FF000E80050B1D2F8E400E946834215D000235E
:1010000082F8E830C2F8E030CD466368574A9B0A60
:10101000013313816CE729462046FFF789FD67E716
:1010200029462046FFF7F0FD62E7B2F8EC803B600E
:1010300008F1030A4FEA9A0A4FEA8A02D11DC90849
:10104000A9EBC1039D46EB460021584600F02EFB5C
:1010500005F1EE0142465846214400F015FB3B687D
:1010600013B9012000F0C4FA94F8D20000F0CAFAD3
:10107000054630B9207200F0E5FA284600F0B8FACB
:10108000C2E7D4F8D4303BB994F8D200B4F8F031C8
:10109000834201D8FFF7E2FED4F8D43043449D42A6
:1010A00008D294F8D200B4F8F0310130834201D86C
:1010B000FFF7D4FE594660685FFA8AF200F0FEFA44
:1010C00008B9CD4689E7636894F8D2004344636069
:1010D000D4F8D43008EB030AC4F8D4A000F092FA94
:1010E000824509D394F8D230D4F8D4000133401BA0
:1010F00084F8D230C4F8D400B8F1FF0F0FD800251F
:10110000257200F09FFA284600F072FA00F03EFDCA
:10111000164B188108B9FFF791FCCD46E8E64FF46D
:101120008A727B6894F8D90002FB0343D3F8E42069
:1011300083F8E86002F58072C3F8E060C3F8E42049
:10114000FFF7B4FDFFF702FE84F8D960B9E700BFEE
:10115000482100204521002000ED00E00400FA05B0
:101160007C210020CDCCCC3D6666663F341100204A
:10117000014B1870704700BF4011002030B54FF090
:101180000054254B226885B09A4207D002F020FB1C
:101190000446C0B90024204605B030BD0025627D5C
:1011A0001E4B1F481A70237DC92203721D49C0F8C7
:1011B000E450093000F068FA2046E022294600F0A9
:1011C00075FA0124E7E7184A184DD36943F0007314
:1011D000D361AA6D164B9A42DCD12B6E013B7E2B5C
:1011E000D8D8144A01AB07CA83E807001846032180
:1011F00000F09CFC6B6D83424FF00003CAD12A6D56
:101200008A4203BFAB652A6E044B1C4601BF1A70AD
:10121000EA6D094B1A60BEE79AAD44C54011002043
:101220007C210020160000200010024000660040D3
:101230005041A0B058660040181100202DE9F0433D
:1012400085B000F0A3FC0223494C63710023029394
:10125000484B2081D3F800C0BCF57A7F12D3464FAB
:10126000464BB7FBFCF59C458CBF0A231123B5FB0D
:10127000F3F603FB1652591EC8B2002A3ED00229CB
:101280000B46F4D89DF80B303D495A1E9DF80A30A4
:101290003C48013B1B0443EA0253BDF80820013AD5
:1012A00013434B6001F0F4FE00230193364B3749A2
:1012B00000934FF48052364B364800F06BFF364BAC
:1012C000197811B1334800F08FFF00F0F3FC0546A8
:1012D000FFF706FC4FF4C873B0FBF3F202FB1303F5
:1012E00005F516709BB218442C4B186002F066FA94
:1012F00008B10F23238105B0BDE8F083731EB3F559
:10130000806FBFD24FF47A75C0EBC00E0EF10303AD
:101310004FEAE30909FB0555C3F3C703C11AC9B274
:1013200009F101088844B5FBF8F5B5F5617F08D9E6
:101330000EF1FF33C3F3C703C11A581E0F28C9B2F9
:1013400014D84A1E072A8CBF00220122581800FB1D
:101350000660B7FBF0F7BC4594D1002A92D0ADF8F7
:1013600008608DF80A308DF80B108BE71346EDE717
:101370003411002018110020005125023F420F00B7
:1013800010110020A8230020D50D000844110020D2
:10139000A10E00084C21002040110020482100200F
:1013A0002DE9F04F80A7D7E900670FF20429D9E9AA
:1013B0000089734D93B00DF1300AFFF7C7FC182276
:1013C0000021504600F072F9DFF8B8B16E4C0023EE
:1013D00052461946584601F093FE014650BB102272
:1013E00008A800F063F9E36883F01003E36000F0FD
:1013F00063FC0DF1240C0B4612A9024611E903000F
:101400008CE803009DF83410C1F30300890649BF3E
:101410000E99BDF83810C1F31C0141F0004158BFCE
:10142000C1F30A018DF82C000891284608A901F0A3
:1014300097F9CCE7284600F0DFFE0446002847D1A4
:1014400000F038FCDFF844B1DBF8003098423FD3BD
:1014500000F030FC0790FFF743FB4FF4C873B0FB7C
:10146000F3F101FB1300079A83B202F516701844DA
:10147000CBF80000DFF818B18DF820409BF8001081
:1014800011B901238DF8203050460791FFF740FB3A
:1014900007990DF12100C1F11004E4B2062C28BF18
:1014A00006245144224600F0EFF808AB03931823BA
:1014B0000293384B013401930123E4B20093324686
:1014C0003B462846049400F0DDFE00238BF80030F4
:1014D00000F0F0FB304A314C1368C31AB3F57A7F41
:1014E00030D3106000F0E8FB02460B46284600F0BF
:1014F00061FF284600F080FE20B3237ADFF8A0B019
:10150000002B14BF032302238BF8053000F0D2FB1D
:101510004FF47A73B0FBF3F00122CBF80000514690
:10152000584600F0B5F9182302931E4B80B2019380
:1015300040F25513CDE903A0009342464B4628469E
:1015400000F0A0FE237ABBB100F0B4FB94F8E830C1
:1015500073B9D4F8E03043B1C01A2368FA2B38BF0E
:10156000FA230533B0EB430F02D30020FFF79EFBB5
:10157000237A002B7FF41FAF13B0BDE8F08F00BFBC
:101580004C210020A8230020000801404821002011
:101590004521002044210020702300207C210020D0
:1015A0003411002074230020401DA12026812A0B25
:1015B000F1C6A7C1D068080F7047000070B501F0F0
:1015C00095FF0024084E094D3080286833888342F7
:1015D00008D901F087FF2B6804440133B4F5C84FE4
:1015E0002B60F2D370BD00BFA4230020782300201D
:1015F00002F00AB800F10060920000F5C84001F066
:10160000AFBF0000054B1A68054B1B889B1A83422D
:1016100002D9104401F066BF0020704778230020F3
:10162000A4230020024B1B68184401F061BF00BFD7
:1016300078230020024B1B68184401F06BBF00BFE9
:1016400078230020064991F8243033B10023082282
:10165000086A81F82430FFF7CDBF0120704700BF32
:101660007C230020022802BF1022014B1A61704720
:1016700000080140022802BF4FF48012014B1A619A
:10168000704700BF00080140002310B5934203D00B
:10169000CC5CC4540133F9E710BD00000346024698
:1016A000D01A12F9011B0029FAD1704703460244EF
:1016B000934202D003F8011BFAE770472DE9F84383
:1016C0001F4D144695F824200746884652BBDFF884
:1016D00070909CB395F824302BB92022FF21484606
:1016E0002F62FFF7E3FF95F824004146C0F108029E
:1016F000A24228BF224605EB8000D6B29200FFF737
:10170000C3FF95F82430A41B1E44F6B2082E1744DC
:101710009044E4B285F82460DBD1FFF793FF002802
:10172000D7D108E02B6A03EB82038342CFD0FFF7C7
:1017300089FF0028CBD10020BDE8F8830120FBE71A
:101740007C2300202DE9F0470D46044600219046F9
:10175000284640F27912FFF7A9FF234620220021F4
:10176000284600F09FFF022220212846231D00F07A
:1017700099FF032222212846631D00F093FF0322D4
:1017800025212846A31D00F08DFF10222821284680
:1017900004F1080300F086FF08223821284604F1EE
:1017A000100300F07FFF08224021284604F11103B6
:1017B00000F078FF08224821284604F1120300F0C7
:1017C00071FF20225021284604F1140300F06AFF23
:1017D00040227021284604F1180300F063FF08221C
:1017E000B021284604F1200300F05CFF0822B82154
:1017F000284604F1210300F055FFC02604F122071A
:101800003B46314608222846083600F04BFFB6F525
:10181000A07F07F10107F3D108223146284604F1E1
:10182000320300F03FFF002704F1330A94F832300E
:101830004FEAC7099F4209F5A47615D3B8F1000F06
:1018400008D131460722284604F5997300F02AFF93
:1018500009F24F16274694F832213B1B93420CD3D2
:10186000F01DC008BDE8F0870AEB070308223146E7
:10187000284600F017FF0137D8E7314607F2331347
:101880000822284600F00EFF08360137E3E7000083
:1018900038B50C460021054621600346C4F8031004
:1018A0002046202200F0FEFE20462B1D0222202191
:1018B00000F0F8FE20466B1D0322222100F0F2FE0C
:1018C0002046AB1D0322252100F0ECFE204610220D
:1018D000282105F1080300F0E5FE072038BD0000CF
:1018E0000023F7B50E460546047F072200911946EE
:1018F00000F09AFD731C0093012200230721284663
:1019000000F092FDC4B9B31C0093052223460821C0
:10191000284600F089FD0D243746B278BB1B934260
:1019200011D32B7FE01DC008AC8ABBB9A04294BF85
:101930000020012003B0F0BDAB8A0824DB00083B87
:10194000DB08B370E8E7FB1C214600930822002364
:10195000284600F069FD08340137DEE7001B18BF98
:101960000120E7E70023F7B50E46047F0822009127
:101970001946054600F058FD731CC4B908220093AF
:1019800011462346284600F04FFD102401237278AB
:101990005F1C013B934211D32B7FE01DC008AC8A32
:1019A000BBB9A04294BF0020012003B0F0BDAB8AB8
:1019B0000824DB00083BDB087370E7E7F3192146D6
:1019C000009308220023284600F02EFD08343B46F1
:1019D000DDE7001B18BF0120E7E70000F8B50E4661
:1019E00005461446002181223046FFF75FFE2B4654
:1019F00008220021304600F055FE7CB9072208215C
:101A000030466B1C00F04EFE0F2401236A785F1CE9
:101A1000013B934204D3E01DC008F8BD0824F4E75D
:101A20002146EB190822304600F03CFE08343B46C4
:101A3000ECE70000F8B50E46054614460021CE221C
:101A40003046FFF733FE2B4628220021304600F0B7
:101A500029FE7CB908222821304605F1080300F050
:101A600021FE30242F462A7A7B1B934204D3E01DAB
:101A7000C008F8BD2824F5E7214607F1090308222C
:101A8000304600F00FFE08340137ECE7F7B5047F6D
:101A90000E460091012310220021054600F0C4FCEF
:101AA000C4B9B31C0093092223461021284600F034
:101AB000BBFC192437467288BB1B9A4211D82B7F76
:101AC000E01DC008AC8ABBB9A04294BF0020012031
:101AD00003B0F0BDAB8A1024DB00103BDB08738041
:101AE000E8E73B1D2146009308220023284600F02A
:101AF0009BFC08340137DEE7001B18BF0120E7E735
:101B000030B5094D0A4491420DD011F8013B5840BF
:101B1000082340F30004013B2C4013F0FF0384EA48
:101B20005000F6D1EFE730BD2083B8ED4FF0FF3322
:101B3000F7B500EB81061946DFF848C0DFF848E04A
:101B4000B0421BD050F8042B01AF0192042217F8C9
:101B5000014B81EA046108240D46DB184941013C30
:101B6000002DBCBF83EA0C0381EA0E0114F0FF04D0
:101B7000F2D1013A12F0FF02E9D1E1E7D843C943BB
:101B800003B0F0BD9336EAA9EBE1F042F7B56B463E
:101B9000354A106851686A4603C3082333493448FC
:101BA00002F0C2F8044690BB0A256B46314A106821
:101BB00051686A4603C308232F492D4802F0B4F840
:101BC0000446002847D00369B3F5CE3F43D8B0F8A8
:101BD0006620B2F57A7F3ED1284A024402F15C01C8
:101BE0008B4238D35C3B224900209E1AFFF788FFC6
:101BF00007463246002004F16401FFF781FFA36825
:101C00009F4228D1E368984208BF002523E003697A
:101C1000B3F5CE3F26D8428BB2F57A7F20D1174A52
:101C2000024402F110018B4218D3103B10490020EE
:101C30009D1AFFF765FF06462A46002004F11801A9
:101C4000FFF75EFFA3689E4202D1E368984201D08D
:101C50000D25AAE70025284603B0F0BD1025A4E70E
:101C60000C25A2E70B25A0E7983D0008DC9B0100AE
:101C700000640008A13D0008909B0100089CFFF74C
:101C8000EFF30983EFF30583014B9B6BFEE700BF86
:101C900000ED00E008B5FFF7F3FF0000EFF3098364
:101CA000EFF30583014B5B6BFEE700BF00ED00E047
:101CB000FEE7000001F0E2BC01F0BABC2DE9F04102
:101CC000456A15B94162BDE8F0814B68AC4623F026
:101CD0006047C3F38A4616EA230638BF3E464FEAFA
:101CE000D37EC3F380782B465A68BEEBD27F22F0B6
:101CF00060440AD0002A18DAA40CB44217D19D42DD
:101D00000FD10D60DEE71346EEE7A74207D102F0E0
:101D10008044C2F3807242450BD054B1EFE708D241
:101D2000EDE7CCF800100B60CDE7B44201D0B4422F
:101D3000E5D81A689C46002AE5D11960C3E700007F
:101D40002DE9F0474FF47F49089D01F007044FEA61
:101D5000D508224405F0070500EBD100944201D1DB
:101D6000BDE8F08704F0070705F0070A57453E462F
:101D700038BF5646111BC6F108068E4228BF0E46D4
:101D8000E108415C08EBD50E13F80EC0B94029FA02
:101D900006F721FA0AF1FFB28CEA010147FA0AF7C5
:101DA00039408CEA010C03F80EC034443544D5E7C1
:101DB000082341F2210280EA012001B240000029FB
:101DC00080B203F1FF33B8BF504013F0FF03F4D1EA
:101DD0007047000038B50C468D18A54200D138BDBB
:101DE00014F8011BFFF7E4FFF7E700000346406823
:101DF00048B1026899895A605A89013292B2914277
:101E00005A8138BF9A81704770B504460D4688B034
:101E1000202200216846FFF749FC20460495FFF781
:101E2000E5FF024658B16B46054608AE1C4603CC9A
:101E3000B44228606960234605F10805F6D11046D2
:101E400008B070BD082817D909280CD00A280CD072
:101E50000B280CD00C280CD00D280CD00E2814BF49
:101E60004020302070470C2070471020704714200D
:101E7000704718207047202070470000082817D9A5
:101E80000C280CD910280CD914280CD918280CD9D6
:101E900020280CD930288CBF0F200E207047092035
:101EA00070470A2070470B2070470C2070470D20A8
:101EB000704700002DE9F843078C0446072F1ED910
:101EC000D0E9029800254FF6FF73C5F12006A5F171
:101ED000200029FA05F108FA06F628FA00F0314345
:101EE0000143C9B21846FFF763FF0835402D03468A
:101EF000EBD13A46E169BDE8F843FFF76BBF4FF617
:101F0000FF70BDE8F883000010B54B6823B9CA8A9A
:101F100063F30902CA8210BD04691A681C60036178
:101F2000C38A013BC3824A60EFE700002DE9F84F06
:101F30001D46CB8A0F46C3F3090105298146924607
:101F40000B4630D00020AAB207F11A049EB2042E2C
:101F50001FFA80F80FD8904503F1010306D3FB8ADE
:101F60000A4462F309030120FB821AE01AF80060B8
:101F70000130E654EAE79045F1D21C23A1F1050BAC
:101F8000BBFBF3F203FB12BB7C681FFA8BF6002C41
:101F900045D14846FFF72AFF044638B978606FF00C
:101FA0000200BDE8F88F4FF00008E6E70026066063
:101FB00078604FF0000BADB2454510D90AEB08032D
:101FC000221D13F8011B08F101089155B1B21B291C
:101FD0001FFA88F82BD0454506F10106F1D8FB8A97
:101FE000C3F30902154465F30903BCE71C4601323B
:101FF00092B22368002BF9D16B1F0B441C21B3FB59
:10200000F1F301339BB29A42D3D2BBF1000FD0D18E
:102010004846FFF7EBFE20B9C4F800B0BFE7012245
:10202000E7E7C0F800B05E4620600446C1E74545DA
:10203000D5D94846FFF7DAFE08B92060AFE7C0F807
:1020400000B0002620600446B6E700002DE9F74FF7
:102050001C465B69074688460092002B00F097807B
:10206000238C2BB1E269002A00F09180072B33D832
:1020700007F10C00FFF7BAFE054628B96FF002051C
:10208000284603B0BDE8F08F14220021FFF70EFBB5
:10209000228CE16905F10800FFF7F6FA208C48F080
:1020A0000041013080B2FFF7E9FEFFF7CBFE0138B7
:1020B00080B22084013028746369228C1B782A4402
:1020C00003F01F0363F03F0313723846696029462B
:1020D000FFF7F4FD0125D3E74FF000094FF0800A28
:1020E0004E464D4600F10C0301930198FFF77EFE2A
:1020F00083460028C2D014220021FFF7D7FA002E11
:102100003BD10222009BABF808300BF1080E1FFAFE
:1021100082FC0CF10100BCF1060F218C80B201D8C9
:102120008E422CD3FFF7AAFEFFF78CFE8E4208BF2B
:102130004FF0400A62690138127880B202F01F0243
:1021400042EA49120BEB00014AEA020A013048F068
:10215000004281F808A08BF8100059463846CBF8A9
:102160000420FFF7ABFD238C0135B3424FF0000A8A
:102170002DB289F00109B8D182E70022C5E7E169F3
:10218000895D01360EF80210B6B20132BFE76FF07A
:10219000010575E7F8B5044615460E4630220021C4
:1021A0001F46FFF783FA069BB5F5001F6360079B88
:1021B00028BF4FF6FF72A3624FF0000338BF6A09D1
:1021C000A760E66197B204F110009A4206D8002396
:1021D0000360A782E3822383E360F8BD06600133D6
:1021E00030462036F1E7000003781BB94BB2002BD4
:1021F000C8BF01707047000000787047F8B50C4602
:10220000C969074611B9238C002B37D1257E1F2DB4
:1022100034D8387828BB228C072A2CD8268A36F066
:1022200003032BD14FF6FF70FFF7D4FD4FF6FF727B
:1022300020F001003602400446EA0565400C45EAFC
:102240004025234629463846FFF700FF002807DDD2
:10225000626913780133DBB21F2B88BF0023137030
:10226000F8BD218A2D0645EA012505432046FFF7E2
:1022700021FE0246E5E76FF00300F1E76FF0010091
:10228000EEE7000070B504461D4616468AB02822C7
:1022900000216846FFF70AFABDF838306946ADF804
:1022A00010300F9B204605939DF84030CDE9026524
:1022B0008DF81830119B0793BDF84830ADF82030E9
:1022C000FFF79CFF0AB070BD2DE9F041D3690546C8
:1022D0000C4616460BB9138C5BBB377E1F2F28D8D4
:1022E00095F80080B8F1000F26D03046FFF7E2FDE8
:1022F0003378210241EAC33141EA0801338A41EAD5
:10230000076141EA034102463346284641F0800115
:10231000FFF79CFE00280ADD3378012B07D1726994
:1023200013780133DBB21F2B88BF00231370BDE885
:10233000F0816FF00100FAE76FF00300F7E70000AB
:10234000F0B504460D461E4617468BB028220021E4
:102350006846FFF7ABF99DF84C3029465A1E5342A8
:1023600053418DF800309DF840306A46ADF810308A
:10237000119B204605939DF84830CDE902768DF8F3
:102380001830149B0793BDF85430ADF82030FFF798
:102390009BFF0BB0F0BD0000406A00B104307047F5
:1023A000436A1A68426202691A600361C38A013B88
:1023B000C38270472DE9F041D0F8208014461D46B5
:1023C00041460027174E09B9BDE8F081D1E9022343
:1023D000A21A65EB0303964277EB03031ED2036A4E
:1023E0008B420DD1FFF790FD036A1B6803620369FE
:1023F0000B60C38A0161016A013B8846C382E2E740
:10240000FFF782FD0B68C8F8003003690B60C38AD0
:102410000161013BC382D8F80010D4E788460968FF
:10242000D1E700BF80841E002DE9F04F8BB00D4630
:1024300014469B468046DDF85090002800F01A8133
:10244000B9F1000F00F01681531E3F2B00F21281EC
:10245000012A03D1BBF1000F40F00C810023CDE92C
:102460000833B8F81430B5EBC30F4FEAC30703D3F2
:1024700000200BB0BDE8F08F2B199F42D8F80C302C
:1024800036BF7F1B2746FFB21BB9D8F81030002B90
:102490007BD0272D4ED8C5F12806B7424FF0000358
:1024A00034BF3E46F6B2009329463246D8F80800BB
:1024B00008ABFFF745FCA7EB060A35445FFA8AFA3A
:1024C0002821B8F8143003F10053053BDB000493D6
:1024D000D8F80C300393039B13B1BAF1000F2CD141
:1024E000D8F8100040B1BAF1000F05D0524600965E
:1024F00008AB691AFFF724FC38B2002FB8D0660782
:102500000AD00AAB03EBD40111F8083C624202F096
:102510000702134101F8083C082C3DD9102C40F269
:10252000B680202C40F2B880BBF1000F00F09D80F7
:10253000082335E0BA460026C2E7049BE02B28BFFB
:10254000E02306930B44AB42059315D95A1B9245E1
:1025500038BF5246039828BFD2B20096691A08AB1A
:1025600004300792FFF7ECFB079A1644AAEB020A25
:102570001544F6B25FFA8AFA049B069A05999B1AEB
:102580000493039B1B680393A5E700933A462946EF
:10259000D8F8080008ABADE7BBF1000F13D001235A
:1025A000B4EBC30F6CD0082C12D89DF82030621EFB
:1025B00023FA02F2D50706D54FF0FF3202FA04F4EF
:1025C00023438DF820309DF8203089F8003050E703
:1025D000102C12D8BDF82030621E23FA02F2D10767
:1025E00006D54FF0FF3202FA04F42343ADF8203051
:1025F000BDF82030A9F800303BE7202C0FD808990F
:10260000631E21FA03F3DA0705D54FF0FF3202FA11
:1026100004F40C430894089BC9F8003029E7402CC7
:102620002BD0DDE90865611EC4F12102A4F121036C
:1026300026FA01F105FA02F225FA03F311431943D0
:10264000CB0712D50122A4F12003C4F1200102FA24
:1026500003F322FA01F1A240524243EA010363EB81
:10266000430332432B43CDE90823DDE90823C9E9BD
:102670000023FEE66FF00100FBE66FF00800F8E6CD
:10268000082CA0D9102CB3D9202CEED8C3E7BBF16D
:10269000000FADD0022383E7BBF1000FBBD00423B2
:1026A0007EE70000012A30B5144638BF012200251C
:1026B000402A28BF402285B0012CCDE9025517D809
:1026C0001B788DF8083053070AD004AB03EBD20512
:1026D00015F8083C544204F00704A34005F8083CF0
:1026E0000346009102A80021FFF72AFB05B030BD88
:1026F000082CE5D9102C03D81B88ADF80830E2E788
:10270000202C02D81B680293DDE7D3E90045CDE910
:102710000245D8E710B5CB681BB98B600B618B8283
:1027200010BD04691A681C600361C38A013BC3823F
:10273000CA60F0E703064CBFC0F3C0300220704708
:1027400008B50246FFF7F6FF022806D15306C2F38A
:102750000F2001D100F0030008BDC2F30740FBE7E2
:102760002DE9F04F93B0CDE903230A6804461046E3
:10277000FFF7E0FF02280CBF0026C2F30626002A5E
:102780000D46824680F2F98112F0C04940F0F58191
:10279000097B002900F0F181022803D02378B3429D
:1027A00040F0EE81C2F304631046069302F07F030B
:1027B0000593FFF7C5FF059B00224FEA83480023DE
:1027C00048EA0A48294448EA4668CE78CDE9082311
:1027D000F309834648EA0008029367D0059B024646
:1027E000009320465346676808A9B847002800F0C0
:1027F000CA81276A4FB9414604F10C00FFF704FB78
:10280000074690B96FF0020054E03B6998450DD03F
:102810003F68002FF9D1414604F10C00FFF7F4FAAC
:1028200007460028EED0236A3B60276297F817C05E
:1028300006F01F08CCF3840CACEB08001FFA80FEF6
:102840000028B8BF0EF12000A8EB0C031FFA83FE8E
:10285000B8BF00B2002B0793BEBF0EF120031BB21E
:102860000793D7E9022152EA010338D04FF0000C58
:10287000039BDFF8F8E19A1A049B63EB010196458C
:102880007CEB01032BD36B7B97F81AE0734519D1CE
:10289000029B002B78D0012821DC7868F8B9DFF89A
:1028A000D0C1944570EB010316D337E0276A27B9EE
:1028B0006FF00C0013B0BDE8F08F3B699845B5D0C0
:1028C0003F68F4E76A4890427CEB010301D30020A3
:1028D000F0E7029B002BFAD0079B0F2B17DCFA7D49
:1028E000B30002F0030203F07C031343FB75394687
:1028F0002046FFF709FB6B7BBB76029B3BB9FB7D58
:10290000C3F38402013262F38603FB75D0E76A7B6E
:10291000BB7E9A42DBD1029B002B35D0B309022B40
:1029200032D0039B1422BB60049B0021FB600DA8E6
:10293000FEF7BCFE039B20460A93049BADF83EB015
:102940000B932B1D0C932B7B8DF840A0013BDBB22E
:10295000ADF83C30069B8DF841808DF84230059BE8
:102960000AA98DF8433094F82C3083F001038DF8D8
:102970004430A3689847FB7DC3F38403013303F01D
:102980001F039B02FB82A2E7FB7DC6F34012B2EB62
:10299000D31F40F0FB80C3F38403434540F0F9802C
:1029A000029A2B7BB609002A4DD0F20762D4032B82
:1029B00040F2F280039BAE1DBB60049B3246FB607D
:1029C0002B7B3946033BDBB204F10C00FFF7AEFA78
:1029D00000280CDA39462046FFF796FAFB7DC3F350
:1029E0008403013303F01F039B02FB820AE7AB88D9
:1029F000DDE908843B834FF6FF73C9F12000A9F19C
:102A0000200228FA09F104FA00F0014324FA02F244
:102A100011431846C9B2FFF7CBF909F10809B9F11A
:102A2000400F0346E9D13146B8822A7B033AD2B23D
:102A3000FFF7D0F9FB7DB882DA43C2F3C01262F32C
:102A4000C713FB7543E7AEB92E1D013B324639462D
:102A5000DBB204F10C00FFF769FA0028BADB2A7B2D
:102A60003146013AB88AD2B2E2E700BF80841E0044
:102A700040420F00F98A013BC1F309010429DAB28F
:102A80005DD80023281D07F11B069A4208D910F8CB
:102A900001CB013306F801C001310529DBB2F4D1C5
:102AA000934228BF0023039938BF04330A91049945
:102AB00038BFDBB20B9107F11B010C91796838BF6D
:102AC0005B190D910E93FB8AADF83EB0C3F3090379
:102AD0001A44069BADF83C208DF84230059B8DF8DA
:102AE00040A08DF8433094F82C308DF8418083F06D
:102AF00001038DF8443000237B602A7BB88A013AB9
:102B0000291DFFF767F93B8BB882834203D120462A
:102B1000A3680AA9984720460AA9FFF7FBFDFB7D99
:102B2000BA8AC3F38403013303F01F039B02FB82C1
:102B30003B8B9A420CBF00206FF01000BAE67B6816
:102B4000002BADD0052001E033461C301E68002E5E
:102B5000FAD1091A081D2E1D184401EB090CBCF10D
:102B60001B0F5FFA89F39BD89A4299D916F8013B5B
:102B700009F1010900F8013BEFE76FF0090099E660
:102B80006FF00A0096E66FF00B0093E66FF00D0011
:102B900090E66FF00E008DE66FF00F008AE600BF42
:102BA000F0B53F4D3F4FEB6943F00073EB61EB69CC
:102BB0003D4B9B6AD3F800623E4046F00106C3F8E5
:102BC0000062D3F800423C4044EA002444F001048F
:102BD000C3F80042002955D000200646C3F81C0265
:102BE000C3F80402C3F80C02C3F8140203EBC004D8
:102BF00001300E28C4F84062C4F84462F6D10027C0
:102C00004FF0010C9678148816F0010F18BFD3F816
:102C100004E20CFA04F01CBF40EA0E0EC3F804E212
:102C200016F0020F18BFD3F80CE203EBC4041CBF6C
:102C300040EA0E0EC3F80CE2760748BFD3F81462E0
:102C400007F1010744BF0643C3F814625668B9424E
:102C5000C4F84062966802F10C02C4F84462D3F8EA
:102C60001C4240EA0400C3F81C02CBD1D3F8002276
:102C700022F00102C3F80022EB6923F00073EB613C
:102C8000EB69F0BD0122C3F84012C3F84412C3F847
:102C90000412C3F81412C3F80C22C3F81C22E5E78F
:102CA000001002400000FFFFA8230020184A08B5CA
:102CB000916A8B688B6013F0010104D013F00C0F44
:102CC00018BF4FF48031D80506D513F4406F14BFF8
:102CD00041F4003141F00201D80306D513F4402F2E
:102CE00014BF41F4802141F00401D3690BB10848BD
:102CF0009847302383F311880021064800F048FBF1
:102D0000002383F31188BDE8084000F099BD00BF9F
:102D1000A8230020B023002038B5124CA36ADD6838
:102D2000AA0712D05A6922F002025A61A36913B1AC
:102D3000012120469847302383F3118800210A4857
:102D400000F026FB002383F31188EB0606D5102143
:102D5000A36AD960236A0BB102489847BDE838409E
:102D600000F06EBDA8230020B823002038B5124C17
:102D7000A36A1D69AA0712D05A6922F010025A618B
:102D8000A36913B1022120469847302383F31188A9
:102D900000210A4800F0FCFA002383F31188EB06B7
:102DA00006D51021A36A1961236A0BB1024898471E
:102DB000BDE8384000F044BDA8230020B82300201F
:102DC00038B50F4CA36A5D682A075D600AD50422F6
:102DD00022701A6822F002021A60636A13B100219D
:102DE000204698476B0706D5A36A9969236A13B1F1
:102DF000034809049847BDE8384000F021BD00BFF2
:102E0000A823002010B50E4C204600F02FF90D4BE2
:102E10000B211320A36200F009F90B21142000F00C
:102E200005F90B21152000F001F90B21162000F007
:102E3000FDF8BDE8104000220E201146FFF7B0BE9D
:102E4000A8230020006400400F4B10B598420446B0
:102E500005D10E4BDA6942F00072DA61DB690122BA
:102E6000A36A1A60A36A5A68D20707D562685168D4
:102E70001268D9611A60064A5A6110BD0121082002
:102E800000F0B0F9EEE700BFA823002000100240D8
:102E90005B87010003291AD8DFE801F0020A0F144A
:102EA000836A9B6813F0E05F14BF01200020704725
:102EB000836A9868C0F380607047836A9868C0F33B
:102EC000C0607047836A9868C0F300707047002044
:102ED0007047000010B5032927D8DFE801F002276A
:102EE0002B2F836A9968C1F30161183103EB011339
:102EF0001078840648BF5468C0F3001158BF948806
:102F00004FEA410148BF41EAC40100F00F00586098
:102F100048BF41F00401906858BF41EA4451D2686B
:102F200041F001019860DA60196010BD836A03F511
:102F3000C073DDE7836A03F5C873D9E7836A03F5D5
:102F4000D073D5E701290AD002290FD081B9836A4D
:102F5000DA68920701D1186903E001207047836A9B
:102F6000D86810F0030018BF01207047836AF2E7A9
:102F70000020704710B539B9836AD96889071BD119
:102F80001B699C0704D110BD012915D00229FAD173
:102F9000816AD1F8C031D1F8C441D1F8C8011061BB
:102FA000D1F8CC015061202008610869800717D151
:102FB000486940F0100012E0816AD1F8B031D1F8D0
:102FC000B441D1F8B8011061D1F8BC0150612020A2
:102FD000C860C868800703D1486940F002004861B2
:102FE000C3F34000C3F38001000140EA41111079AE
:102FF00020F030000143117189064BBF916811899F
:10300000DB085B0D4CBF63F31C0163F30A0113790A
:1030100048BF916064F3030313714FEA14234FEA2E
:10302000144458BF118113705480ACE70122090188
:1030300000F1604303F56143C9B283F8001300F067
:103040001F039A4043099B0003F1604303F561436A
:10305000C3F880211A607047090100F16040C9B2CD
:1030600000F56D4001767047FFF7CCBE0123037079
:10307000002300F10802C0E9022200F11002C0E9B9
:103080000422C0E90633C0E90833436070470000FA
:1030900010B53023044683F3118802234160037086
:1030A000FFF7D2FE04230020237080F3118810BDA7
:1030B0002DE9F0411F4604460D461646302383F3A2
:1030C000118800F108082378052B0DD029462046E9
:1030D000FFF7E0FE40B1204632462946FFF7FAFEF0
:1030E000002080F3118808E03946404600F040F99E
:1030F0000028E8D0002383F31188BDE8F0810000A8
:103100002DE9F0411F4604460D461646302383F351
:10311000118800F110082378052B0DD02946204690
:10312000FFF710FF40B1204632462946FFF722FF45
:10313000002080F3118808E03946404600F018F975
:103140000028E8D0002383F31188BDE8F081000057
:1031500000238268037503691B6899689142FBD25A
:103160005A680360426010605860704700238268AC
:10317000037503691B6899689142FBD85A6803601C
:10318000426010605860704708B50846302383F3EA
:1031900011880B7D032B05D0042B0DD02BB983F3A5
:1031A000118808BD00228B691A604FF0FF338361DC
:1031B000FFF7CEFF0023F2E7D1E9003213605A6037
:1031C000F3E70000FFF7C4BF054BD968087518681E
:1031D000026853601A6001220275D860FDF796BB41
:1031E000D823002030B50C4B0446DD684B1C87B05B
:1031F0000FD02B466846094A00F0F0F82046FFF74A
:10320000E3FF009B13B1684600F0F0F8A86907B02F
:1032100030BDFFF7D9FFF9E7D82300208931000836
:10322000044B1A68DB6890689B68984294BF002042
:1032300001207047D8230020084B10B51C68D868BF
:10324000226853601A6001222275DC60FFF78EFF4E
:1032500001462046BDE81040FDF758BBD8230020AA
:10326000044B1A68DB6892689B689A4201D9FFF7A1
:10327000E3BF7047D823002038B501230025064C52
:10328000064907482370656000F020FB0223237085
:1032900085F3118838BD00BF30250020B03D0008FF
:1032A000D823002000F0B4B8EFF3118020B9EFF379
:1032B0000583302282F311887047000010B530B9C1
:1032C000EFF30584C4F3080414B180F3118810BD32
:1032D000FFF7C6FF84F31188F9E700008B60022333
:1032E00008618B82084670478368A3F1440243F863
:1032F000142C026943F8442C426943F8402C094AD3
:1033000043F8242CC268A3F1200043F8182C0222B1
:1033100003F80C2C002203F80B2C034A43F8102C62
:10332000704700BF1D090008D823002008B5FFF72B
:10333000DBFFBDE80840FFF745BF0000024BDB683C
:1033400098610F20FFF740BFD8230020302383F37C
:103350001188FFF7F3BF000008B50146302383F35F
:1033600011880820FFF73EFF002383F3118808BD72
:10337000064BDB6839B1426818605A6013604360DD
:103380000420FFF72FBF4FF0FF307047D8230020F5
:1033900038B504460D462068844200D138BD036824
:1033A00023605C608561FFF70DFFF4E710B50A4C00
:1033B00023699A6891420CD85A6881600360426020
:1033C00010609A685860511A99604FF0FF33A361FA
:1033D00010BD1B68891AECE7D8230020C0E903233D
:1033E000002310B410BC4361FFF7E0BF036881689D
:1033F0009A680A449A60426813605A6000234FF04A
:10340000FF320360014B9A61704700BFD823002050
:1034100070B5124D2A46EB690133EB6152F8103F4B
:10342000934206D030269A68013A9A602C69A368C4
:1034300003B170BDD4E900210A605160236083F3B9
:1034400011882046D4E90331984786F311886169D1
:103450000029EBD02046FFF7A9FFE7E7D82300209B
:1034600000207047FEE70000704700004FF0FF307B
:1034700070470000BFF34F8F024AD368DB07FCD4CC
:10348000704700BF0020024008B5074B1B7853B9B6
:10349000FFF7F0FF054B1A69120641BF044A5A6054
:1034A00002F188325A6008BD482500200020024001
:1034B0002301674508B5054B1B7833B9FFF7DAFFE1
:1034C000034A136943F08003136108BD48250020B7
:1034D000002002407F289ABF00F5003080020020C3
:1034E000704700004FF480607047000080207047F4
:1034F0007F2808B50BD8FFF7EDFF00F58063026861
:10350000013204D104308342F9D1012008BD0020EA
:10351000FCE700007F2810B504461CD8FFF7AAFF7F
:10352000FFF7B2FFF3220D4B4FF48061DA60022205
:103530001A61FFF7CFFF58611A6942F040021A6121
:10354000FFF798FF00F004F9FFF7B4FF2046BDE84D
:103550001040FFF7CDBF002010BD00BF002002408B
:103560002DE9F843054612F00100144606D040F25A
:10357000F32200201E4B1A60BDE8F8831D4BAA18E9
:103580009A4204D94FF43E72194B1A60F4E7FFF7E0
:103590007BFF4FF00109FFF76DFFDFF85C806D1ACC
:1035A000012C0F4605EB010603D8FFF783FF01202E
:1035B000E2E73B88C8F8109033800020FFF75AFFFD
:1035C000C8F81000338831F8022B9BB29A420CD015
:1035D00040F20F32064B1A60084B1E60084B1C600D
:1035E000084B1F60FFF766FFC6E7023CD8E700BF45
:1035F0004425002000000208002002403825002059
:10360000402500203C250020084908B50B7828B14A
:103610001BB9FFF739FF01230B7008BD002BFCD04D
:10362000BDE808400870FFF745BF00BF48250020EF
:1036300070B5FFF739FE4FF47A710D4B0D4EDB6913
:10364000326801FB03F3934237BF0B4A0A495168C2
:10365000156836BF4C1CD1E9005454605D1944F123
:1036600000043360FFF72AFE2846214670BD00BFE4
:10367000D82300204C2500205025002070B5FFF7EE
:1036800013FE4FF47A710F4B0F4EDB69326801FB6A
:1036900003F3934237BF0D4A0C49516815683ABF8E
:1036A0004C1C5460D1E900545D1944F100043360AE
:1036B000FFF704FE4FF47A72002328462146FCF7F8
:1036C00031FF70BDD82300204C250020502500205C
:1036D00010B5094C013AD2B2FF2A00D110BD5008F2
:1036E00054F82030013054F820009BB243EA0043E4
:1036F00041F8043BEEE700BF046C004010B50748FA
:10370000013AD2B2FF2A00D110BD0C88530840F80C
:1037100023404C88013340F82340F1E7046C00401B
:1037200007B50122002001A9FFF7D2FF019803B0DD
:103730005DF804FB13B50446FFF7F2FFA04205D085
:103740000122002001A90194FFF7D8FF02B010BDAB
:103750007047000045F25552064B1A6002225A602B
:1037600040F6FF729A604CF6CC421A600122024B7E
:103770001A707047003000405C250020034B1B7816
:103780001BB14AF6AA22024B1A6070475C25002042
:1037900000300040044B1A682AB902F1804202F559
:1037A0000432526A1A607047582500204FF0807228
:1037B000014B5A62704700BF0010024008B5FFF786
:1037C000E9FF024B1868C0F3407008BD582500207F
:1037D00008B5FFF7DFFF024B1868C0F3007008BDA3
:1037E00058250020EFF30983203383F30988002351
:1037F00083F3118870470000302080F3118862B68F
:103800000C4B0D4AD96821F4E0610904090C0A4304
:10381000DA60D3F8FC20094942F08072C3F8FC203A
:103820000A6842F001020A602022DA7783F8220057
:10383000704700BF00ED00E00003FA05001000E053
:10384000302310B583F311880B4B5B6813F40063CE
:103850000FD0EFF309844FF08073203CE36184F3D1
:103860000988FFF7DDFC10B1044BA36110BD044BC8
:10387000FBE783F31188F9E700ED00E02F0900086A
:103880003209000870470000FEE700000A4B0B48B1
:103890000B4A90420BD30B4BC11EDA1C121A22F0BA
:1038A00003028B4238BF00220021FDF7FFBE53F810
:1038B000041B40F8041BECE7343E0008E025002020
:1038C000E0250020E0250020FEE7000070B500257F
:1038D00004461A4B86B05860856201630E46FFF7B6
:1038E0008BFF04F11003C4E904334FF0FF33A361ED
:1038F000134BE561D9692B460A462046C4E90823E3
:1039000004F134018023C4E900440E4AA560E56255
:103910002565FFF7E3FC01230B4AE0600375009285
:10392000726868460192B268CDE90223074BCDE97F
:103930000435FFF7FBFC06B070BD00BF302500204A
:10394000D8230020BC3D0008C13D0008C93800084C
:1039500000F030B808B500F063F9FFF78DFCBDE862
:103960000840FFF717BF0000704700004FF0FF311D
:103970000E4B1A6919611A6900221A611869D86810
:10398000D960D968DA60DA68DA6942F08052DA61BF
:10399000DA69DA6942F00062DA61054ADB691368C4
:1039A00043F48073136000F01BB900BF00100240A5
:1039B00000700040194B1A6842F001021A601A6840
:1039C0009007FCD51A6802F0F9021A6000225A60CA
:1039D0005A6812F00C0FFBD11A6842F480321A6058
:1039E0001A689103FCD55A6842F4E8125A601A68C2
:1039F00042F080721A601A689201FCD51221084ABE
:103A00005A60084A11605A6842F002025A605A68C5
:103A100002F00C02082AFAD1704700BF00100240E1
:103A200000641D0000200240084A08B5516913686F
:103A30000B4003F00103536123B1054A13680BB136
:103A400050689847BDE80840FFF7FABE00040140FF
:103A500060250020084A08B5516913680B4003F03F
:103A60000203536123B1054A93680BB1D0689847AC
:103A7000BDE80840FFF7E4BE0004014060250020D7
:103A8000084A08B5516913680B4003F004035361F9
:103A900023B1054A13690BB150699847BDE8084046
:103AA000FFF7CEBE0004014060250020084A08B59B
:103AB000516913680B4003F00803536123B1054AB1
:103AC00093690BB1D0699847BDE80840FFF7B8BECD
:103AD0000004014060250020084A08B551691368B8
:103AE0000B4003F01003536123B1054A136A0BB175
:103AF000506A9847BDE80840FFF7A2BE00040140A5
:103B000060250020174B10B55A691C68144004F456
:103B100078725A61A30604D5134A936A0BB1D06A2E
:103B20009847600604D5104A136B0BB1506B984749
:103B3000210604D50C4A936B0BB1D06B9847E20574
:103B400004D5094A136C0BB1506C9847A30504D5F2
:103B5000054A936C0BB1D06C9847BDE81040FFF755
:103B60006FBE00BF00040140602500201A4B10B555
:103B70005A691C68144004F47C425A61620504D5F9
:103B8000164A136D0BB1506D9847230504D5134A9F
:103B9000936D0BB1D06D9847E00404D50F4A136EB6
:103BA0000BB1506E9847A10404D50C4A936E0BB12B
:103BB000D06E9847620404D5084A136F0BB1506F5A
:103BC0009847230404D5054A936F0BB1D06F9847EB
:103BD000BDE81040FFF734BE00040140602500201E
:103BE000062108B50846FFF721FA06210720FFF74E
:103BF0001DFA06210820FFF719FA06210920FFF710
:103C000015FA06210A20FFF711FA06211720FFF7FF
:103C10000DFABDE8084006212820FFF707BA00008A
:103C200008B5FFF7A3FE054800F00CF8FFF71CFAF3
:103C3000FFF79AFEBDE8084000F002B8C83D000852
:103C400000F042B8002319461C4A0133102BC2E988
:103C5000001102F10802F8D1194B9A6942F07D0275
:103C60009A619B690268174BDA6082685A60426801
:103C70001A60C26803F58063DA6042695A600269BB
:103C80001A608269C3F80C24026AC3F80424C2696A
:103C9000C3F80024426AC3F80C28C26AC3F8042897
:103CA000826AC3F80028026BC3F80C2C826BC3F83D
:103CB000042C426BC3F8002C704700BF6025002025
:103CC00000100240000801404FF0E023044A0821A0
:103CD0005A6100229A6107220B201A61FFF7BCB9D2
:103CE0003F19010008B5302383F31188FFF7DAFA92
:103CF000002383F3118808BD08B5FFF7F3FFBDE883
:103D00000840FFF79DBD000010B501390244904204
:103D100001D1002005E0037811F8014FA34201D042
:103D2000181B10BD0130F2E72DE9F0419BB10446AC
:103D3000C91A1778014403F1FF3C8C42204601D98F
:103D4000002008E005780134BD42F6D10CEB0405F3
:103D5000D618A54201D1BDE8F08115F8018D16F8FD
:103D600001EDF045F5D0E8E7034611F8012B03F823
:103D7000012B002AF9D170476F72672E617264754A
:103D800070696C6F742E663130332D51696F7465B4
:103D90006B5065726970680040A2E4F16468910636
:103DA0000041A3E5F265699207000000633000005E
:103DB000AC3D000830240020302500206D61696E84
:103DC0000069646C65000000001800004444414430
:103DD000445449440100000042444444444444449F
:103DE00000000000444444444444444400000000B3
:103DF0004444444444444444000000004444444493
:103E00004444444450C7FF7F01000000000000000C
:103E1000E803000000000000009C0100000000001A
:103E2000640000000000000040420F00FE2A010074
:043E3000D2040000B8
:00000001FF
